:103DF7000FAA0FA50F9F0F9A0F940F8D0F870F8094
:103E07000F780F710F680F600F570F4E0F450F3B5D
:103E17000F300F250F1A0F0E0F020EF50EE80EDBEF
:103E27000ECC0EBE0EAE0E9F0E8E0E7D0E6C0E5A73
:103E37000E470E340E200E0C0DF70DE20DCB0DB50F
:103E47000D9D0D850D6D0D540D3A0D200D050CE9D9
:103E57000CCE0CB10C940C760C580C3A0C1B0BFBCB
:103E67000BDB0BBB0B9A0B790B570B350B130AF1BB
:103E77000ACE0AAB0A870A640A400A1C09F809D461
:103E870009B0098C09670943091F08FB08D608B25E
:103E9700088E086A0846082307FF07DC07B9079654
:103EA70007730751072F070D06EC06CA06AA0689EE
:103EB70006690649062A060A05EC05CD05B00592EE
:103EC70005750558053C0520050504EA04CF04B52A
:103ED700049C04820469045104390422040B03F48A
:103EE70003DE03C803B2039D038903750361034D12
:103EF700033B03280316030402F202E102D102C0C6
:103F070002B002A0029102820273026502570249BF
:103F1700023C022F02220216020901FD01F201E60C
:103F270001DB01D001C601BB01B101A7019D0194CD
:103F3700018B01820179017001680160015801500C
:103F47000148014101390132012B0125011E0118E8
:103F57000111010B010500FF00FA0ECF0EBB0EA7E2
:103F67000E920E7C0E650E4D0E340E190DFE0DE1F0
:103F77000DC40DA50D850D640D420D1E0CFA0CD454
:103F87000CAE0C860C5D0C330C080BDC0BB00B82F3
:103F97000B540B250AF50AC40A930A610A2F09FD77
:103FA70009CA09960963092F08FC08C8089508611A
:103FB700082E07FB07C8079607640733070206D2D0
:103FC70006A206730645061705EA05BF05930569A8
:103FD7000540051704F004C904A3047E045A0437F6
:103FE700041503F403D303B403960378035B033F79
:103FF7000324030A02F002D702BF02A80292027C3E
:1040070002670253023F022C021A020801F701E677
:1040170001D601C701B801A9019C018E0181017474
:104027000168015D01510146013C01320128011F70
:104037000115010D010400FC00F400EC00E500DEB1
:1040470000D700D000CA00C300BD00B800B200AD61
:1040570000A700A2009E009900940090008C0087A2
:1040670000840080007C007800750072006E006B91
:104077000068006500620060005D005A0058005546
:1040870000530051004E004C004A004800460044CF
:1040970000430041003F003E003C003A0039003732
:1040A70000360035003300320031002F002E002D7E
:1040B700002C002B002A00290028002700260025B5
:1040C7000024002300010C01010502011E030A96CA
:1040D7000401320504040600640701010800000911
:1040E700015A0A01040B00030E01010F000112001F
:1040F7006413010114013C1501FA1664FA17FFFF56
:104107001D00072000072400022632962701012CF4
:10411700000130030332010333000235FFFF36038A
:10412700073CFFFF3DFFFF180002191E461A000259
:104137001B00022D32C82E00012F013CFAFAFA1893
:10414700000019FFFF1A00001B00002D32C82E00C7
:10415700012F013CFAFAFA18000019FFFF1A0000B4
:0F4167001B00002DFFFF2EFFFF2FFFFFFAFAFABC
:10004800E50C90249BF8282873803475E700A210EB
:10005800B34008E5B54408F5B58006E5B554F7F5AD
:10006800B575E710801975E700A210B34008E5B52B
:0F0078004402F5B58006E5B554FDF5B575E71002
:09249B0002005102005302006E20
:100087002290083BE0900041F090083CE090004847
:10009700F090083DE0900049F090083EE090004C59
:1000A700F090083FE090004DF0900840E09000503D
:1000B700F0900841E0900051F0900842E090005C19
:1000C700F0900843E090005EF0900844E0900062F2
:1000D700F0900845E0900064F0900846E0900065D5
:1000E700F0900847E0900066F0900848E0900067BD
:1000F700F0900849E090006AF090084AE090006BA1
:10010700F090084BE090006DF090084CE090006E86
:10011700F090084DE090007AF090084EE090007B58
:10012700F090084FE090007CF0900850E090007D40
:10013700F0900851E090007EF0900852E090007F28
:10014700F0900853E0900080F0900854E090008110
:10015700F0900855E0900083F0900856E0900084F6
:10016700F0900857E0900085F0900858E0900086DE
:10017700F090007AE090002BF090007BE090002C4C
:10018700F090007CE090002DF090007DE090002E34
:10019700F090007EE090002FF090007FE09000301C
:1001A700F0900080E0900031F0900081E090003204
:1001B700F0900083E0900027F0900084E090002802
:1001C700F0900085E0900029F0900086E090002AEA
:1001D700F0744C90010FF07465900110F0747890F2
:1001E7000111F07475900112F07473900113F0749B
:1001F70020900114F07441900115F07436900116A7
:10020700F07435900117F07430900118F074209055
:100217000119F0743590011AF0745390011BF074B2
:100227005090011CF0744490011DF09003BEE090C3
:1002370003FEF022900838E0FEA3E0FF7463BE00DF
:1002470010D39F400C9040CB12001EE493F5998089
:100257004C90000BE0D394044014900838E0FEA3C0
:10026700E0FF9040CB12001EE493F599802F900099
:100277000BE0D394034014900838E0FEA3E0FF900E
:1002870040E312001EE493F5998012900838E0FECF
:10029700A3E0FF9040FB12001EE493F59990083805
:1002A70012000E900838E0FEA3E0FF747B6F4E70DB
:1002B700037566002290005CE0B40105756F02804B
:1002C70003756F01A209B34016900124E0700C90EA
:1002D7000125E07006900126E060028002C20990C5
:1002E7000124E0B4300F900125E0B44708900126BF
:1002F700E0643B60028004D20A8002C20AE549B486
:10030700010280030203D690007AE090002BF09060
:10031700007BE090002CF090007CE090002DF090A6
:10032700007DE090002EF090007EE090002FF0908E
:10033700007FE0900030F0900080E0900031F09076
:100347000081E0900032F0900083E0900027F09069
:100357000084E0900028F0900085E0900029F0905C
:100367000086E090002AF0900063E0B40117900047
:1003770000740FF0A374FFF0900002E4F0A3F07490
:1003870002900063F0900063E0B40341900002E044
:10039700FEA3E0FF900000E0FCA3E0FD1200037461
:1003A700101243467408124338EF900062F0EF7062
:1003B7000674FF900062F07400900063F0900001F3
:1003C700E0900048F0900000E0900049F08009902C
:1003D700006BE070037549017E817F99900041E0D1
:1003E7008E048F05FF1243288C338D3490004DE027
:1003F70075F0FAA4FFAEF090004CE08E048F05FF75
:100407001243288C378D38900039E0F54F9000372C
:10041700E0FE900053E0B50618900036E0FE90002D
:1004270052E0B5060C900035E0FE900043E06E60A8
:100437006F900053E07006900052E06006740090E1
:100447000043F0900053E0B402089000337401F0C9
:100457008005900033E4F0900052E0B40208900069
:10046700347401F08005900034E4F0900052E060AD
:1004770006900034E060028005754F048003754FD5
:1004870005E54AB54902D20B900052E0900036F0DC
:10049700900053E0900037F0900043E0900035F073
:1004A7007401900088F07400900089F07401900046
:1004B7008AF0740090008BF0740090008CF0740048
:1004C70090008DF0740090008EF0740190008FF012
:1004D7007400900090F07400900091F07400900008
:1004E70092F07400900093F07400900094F0740000
:1004F700900095F07401900096F07400900097F0CA
:100507007401900098F07400900099F074009000C6
:100517009AF0740090009BF0740090009CF07401B6
:1005270090034CF0740090034DF0740090034EF06C
:10053700740090034FF07400900350F07400900320
:1005470051F07400900352F0740190038CF0740121
:1005570090038DF0740090038EF0740090038FF079
:100567007400900390F07400900391F0740090036E
:1005770092F074009003CCF074019003CDF07400F6
:100587009003CEF074009003CFF074009003D0F086
:1005970074009003D1F074009003D2F074009004BB
:1005A7000CF0740090040DF0740190040EF07400C8
:1005B70090040FF07400900410F07400900411F090
:1005C7007400900412F0740090044CF074009004CE
:1005D7004DF0740090044EF0740190044FF07400D5
:1005E700900450F07400900451F07400900452F09D
:1005F7001224D722C293C294C291C292C203C204E8
:10060700E5B554FBF5B5754405E54404F54590009B
:1006170039E0F54F900026E4F0C208E5B554FEF541
:10062700B5900026E4F0755200C28E758D00758B6B
:1006370000754100752600752500D28EC296C295B9
:10064700C2A0C297C287E5B554BFF5B5E5B554DF7B
:10065700F5B5E5B554EFF5B5E5B5547FF5B5E5B5B1
:1006670054F7F5B5E5B554FDF5B52275580075573E
:1006770000AE57AF587462BE00039F500302072FA6
:100687009040CB12001EE49390003812435E0FBFD8
:1006970000010EE0FC9040CB12001EECFEE493FF3D
:1006A700EEC39F5026AE57AF580FBF00010E9040C4
:1006B700CB12001EAE57AF58E493FC9040CB12000C
:1006C7001EE49390003812435EECF0AE57AF58909B
:1006D70040CB12001EE49390003812435EE0FC907A
:1006E70040CD12001EECFCE493FDECD39D40199025
:1006F70040CD12001EE493FC9040CB12001EE49301
:1007070090003812435EECF0AE57AF5874022FFFDB
:1007170050010E8E578F587858740126F6500418DA
:10072700E436F6400302067822755800755700AE86
:1007370057AF587417BE00039F50030207FD90413F
:100747002E12001EE49390003812435E0FBF000183
:100757000EE0FC90412E12001EECFEE493FFEEC368
:100767009F5026AE57AF580FBF00010E90412E1273
:10077700001EAE57AF58E493FC90412E12001EE4C2
:100787009390003812435EECF0AE57AF5890412E6D
:1007970012001EE49390003812435EE0FC90413053
:1007A70012001EECFCE493FDECD39D401990413000
:1007B70012001EE493FC90412E12001EE493900059
:1007C7003812435EECF0AE57AF5874126F4E700696
:1007D700755818755700AE57AF5874022FFF500160
:1007E7000E8E578F587858740126F6500418E43641
:1007F700F6400302073622755800755700AE57AF0B
:10080700587417BE00039F50030208CB904146124D
:10081700001EE49390003812435E0FBF00010EE004
:10082700FC90414612001EECFEE493FFEEC39F507E
:1008370026AE57AF580FBF00010E90414612001E5B
:10084700AE57AF58E493FC90414612001EE49390D4
:10085700003812435EECF0AE57AF58904146120095
:100867001EE49390003812435EE0FC90414812006A
:100877001EECFCE493FDECD39D4019904148120017
:100887001EE493FC90414612001EE4939000381238
:10089700435EECF0AE57AF5874126F4E7006755842
:1008A70018755700AE57AF5874022FFF50010E8EC0
:1008B700578F587858740126F6500418E436F640D6
:1008C7000302080422755800755700AE57AF5874D5
:1008D70017BE00039F500302099990415E12001E44
:1008E700E49390003812435E0FBF00010EE0FC90C6
:1008F700415E12001EECFEE493FFEEC39F5026AE4E
:1009070057AF580FBF00010E90415E12001EAE5741
:10091700AF58E493FC90415E12001EE493900038B8
:1009270012435EECF0AE57AF5890415E12001EE4E2
:100937009390003812435EE0FC90416012001EEC79
:10094700FCE493FDECD39D401990416012001EE436
:1009570093FC90415E12001EE49390003812435EB0
:10096700ECF0AE57AF5874126F4E70067558187585
:100977005700AE57AF5874022FFF50010E8E578F96
:10098700587858740126F6500418E436F6400302E6
:1009970008D22212067290F802E493B404051207F3
:1009A700FE801290F802E493D394044005120730B6
:1009B70080031208CC220542220541220543C2CFFB
:1009C7002290F800E4936406600280FE7584017546
:1009D700A70075FF8090083AE4F075C91075A70F56
:1009E70075A1C775A70075D90075CEFF75A70F75D7
:1009F700F1FE75F2FF75F33775F47875A4BA75A52E
:100A0700FF75A60775AE0075AFFF75D48175D5FF65
:100A170075D6FF75D7FFC296C295C2A0C297C2917D
:100A2700C293C294E5B554DFF5B5E5B554EFF5B516
:100A3700E5B5547FF5B5E5B554F7F5B5E5B554FD1E
:100A4700F5B5E5B554FEF5B575A70075A20175A115
:100A57004775F80975BC0175BE0475BD6C75BE0791
:100A670075BDA075BE0875BD0175BC0075BB187551
:100A7700BC2075BA0875E88075D11375A70F75E1A5
:100A87000575E20075C740759700759780740A125F
:100A970043187597C0E5975420700280F8758F0248
:100AA70075A700D2AF75980075A90C75A70F75AB20
:100AB7004375ADFB75AC1E75A700758911758E0062
:100AC700758C00758A00D2A9D28C758D00758B0044
:100AD700D2ABD28E75CD0075CC0075CA0075CB0030
:100AE700D2ADC2CFD2CA7591047592007593CD75F8
:100AF700EF0675D94075CF01900838E4F0A3F0757B
:100B07006600756700C299C20C1205FB7509C875A6
:100B1700080012260D75A70FE5FC900015F0E5FB00
:100B2700900016F0E5FA900017F0E5F9900018F03C
:100B370075A70090F800E493F55612272C122C663F
:100B470090F807E493900022F0900022E044089088
:100B57000022F0900022E054FE900022F01200885C
:100B6700900859E0900124F090085AE0900125F090
:100B770090085BE0900126F0900124E0700C900152
:100B870025E07006900126E060028004C209800219
:100B9700D209754901754A017403900036F01209AC
:100BA7009A7400900063F0740090006CF01202BC1D
:100BB7007406900008F07400900009F07402900029
:100BC7000AF090F802E49390000BF090F803E49396
:100BD70090000CF090F804E49390000DF0740590E9
:100BE700000EF090000BE0B40406740490000EF0C1
:100BF70090000BE0B40306740390000EF0740490A9
:100C0700000FF07403900010F07406900011F07458
:100C170002900012F090F805E493900013F090F81A
:100C270006E493900014F0740090001CF074009098
:100C3700001DF0740090001EF0740090001FF07407
:100C470000900020F07400900021F074FF900023C2
:100C5700F0A2B6B39200A2B3B39201756C00743AD6
:100C6700900738F074FD900739F0C20B900024E428
:100C7700F0754B00752400752300753E00752A003A
:100C8700752900753F007546007547007545017564
:100C970054007553007555CD754800753B00753C7C
:100CA70000753D00753A00753900754E00900004D7
:100CB70074FDF0A374E8F0900024E4F074649000ED
:100CC70025F0C205755100C206754200C2A1C2A235
:100CD700C287C290E5B554BFF5B51225E0C203C27D
:100CE70004D2B0D2B7D2A7D2A6D2B1D2A37E017F07
:100CF70000900049E0124346900048E02FFF500162
:100D07000E900000EEF0A3EFF0EFD394FFEE940FF8
:100D17004007900000E4F0A3F0900062E0700674D2
:100D2700FF900062F0D29CD2EC75CF01A298B3403D
:100D370005C298123012E5666006A299B3B3400265
:100D47008005C299123428E56764016005E567B438
:100D5700040280D5E542D39405400CE54BC394C803
:100D67005002054B754200E555C394F0501A78536D
:100D770012003FAE53AF54EFD394E8EE940340080C
:100D87000555755400755300C28E7E047F00E541FA
:100D9700124346E58D75F004A4FDACF0EF2DFDEE92
:100DA7003CFCE58B75F04084FF7E00ED2FFFEC3EA9
:100DB700FE8E258F26D28EA2B6300001B3500302D5
:100DC7000F2CA2B6300001B35003020F2CA2B6407D
:100DD7007F0546A20C400575FFA0D20CAE39AF3A8D
:100DE7007441BE00039F5006E5B54401F5B5900078
:100DF70025E4F0900041E0C395465052E52645258D
:100E0700600F7C817D99AE25AF261241768E238FA8
:100E170024AE23AF24E53E2FFF50010E7401124389
:100E2700388E238F2485243E754601C28E758D002A
:100E3700758B00754100D28E7403BE00039F500668
:100E47009000267401F0E56CB40D03756C00D200B8
:100E5700A2B6B35003020F2C900025E4F0C2009015
:100E67000055E060077401F508123569900058E0F5
:100E770060077402F508123569E548B40708E5B557
:100E87004480F5B58006E5B5547FF5B5A203B340B8
:100E970004D2878002C287900043E06004D290802A
:100EA70002C290900034E0B40104D2A18002C2A132
:100EB700900033E0B40104D2A28002C2A2A208B318
:100EC7004008E5B54440F5B58006E5B554BFF5B52E
:100ED70090000EE0FE90000BE0C39E400990000BCF
:100EE700E0D39408400974FB900024F01205FB90AE
:100EF700000CE0601590000CE0FE90000AE06E60C8
:100F07000974FC900024F01205FB90000DE06015B9
:100F170090000DE0FE90000FE06E600974FE9000F7
:100F270024F01205FBC2CA7E017F00E54312434647
:100F3700E5CD2FFF50010E8E278F28D2CA9000666D
:100F4700E0B40148900004E0FCA3E0FDEFC39DEE90
:100F57009C4039B207E52A45296013A207B3400828
:100F6700E5B54404F5B58006E5B554FBF5B5900045
:100F770004E0FEA3E0FF900006E0FCA3E0FDEF2DF8
:100F8700FDEE3CFC900004ECF0A3EDF0A2B33001C1
:100F970001B350030210D8A2B3300101B3500302CA
:100FA70010D8A2B350030210D10547A20C40057513
:100FB700FFA0D20CAE39AF3A7441BE00039F500672
:100FC700E5B54401F5B5900025E4F090004CE0C389
:100FD700954740030210CFE5284527600F7CEA7D3F
:100FE70060AE27AF281241768E298F2AAE29AF2A05
:100FF70090004DE012434674FF8E048F05FF1243A5
:10100700288C298D2AE53F2DFD50010C74018C0693
:101017008D071243388E298F2A852A3FA208B340AD
:10102700157464124346900051E08E048F05FF1239
:1010370043288C298D2A754701900004E0FEA3E020
:10104700FFAC27AD28120003900004EEF0A3EFF0E9
:101057007AFF7BFF900065E08A048B05FF12432827
:10106700AE27AF28EDD39FEC9E4023900065E0129A
:10107700434674828E048F05FF124328900067E071
:10108700FF124328900006ECF0A3EDF0802DAE2769
:10109700AF2874828E048F05FF124328900065E005
:1010A7008C068D07124346900067E08E048F05FF7C
:1010B700124328900006ECF0A3EDF0C2CA75CD00EC
:1010C70075CC00754300D2CAD201A2B3B34002C2A5
:1010D70001900026E0B40107E548C39406400302E7
:1010E7001C53E5529024A4F8282873900043E0C3CA
:1010F70094024003021246E544D3940150030212BE
:1011070046E54475F040A4FFAEF09002FC12001EC5
:10111700E0C3953C5018E54475F040A4FFAEF0904D
:1011270002FB12001EE0F52E752D00021246E54463
:1011370075F040A4FFAEF09002FA12001EE0C395CE
:101147003C40030211E2E54475F040A4FFAEF09085
:1011570002FB12001EE54475F040A4FFAEF0E0FC70
:101167009002F912001EECFEE0FFEEC39FFEE5447D
:101177008E0475F040A4FFAEF09002FA12001EE054
:10118700F404253C8C0088F0A4FFAEF0E5448F04FE
:101197008E0575F040A4FFAEF09002FC12001EE52C
:1011A7004475F040A4FFAEF0E0FA9002FA12001E78
:1011B700EAFEE0FFEEC39FFECDCCCD8E071243289B
:1011C700E54475F040A4FFAEF09002F912001EE06E
:1011D7002DFD50010C8C2D8D2E8064E54475F0405B
:1011E700A4FFAEF09002F912001EE54475F040A48A
:1011F700FFAEF0E0FC9002F812001EECFEE0FFEEFE
:10120700C39F853CF0A4FFAEF0E5448F048E0575BF
:10121700F040A4FFAEF09002FA12001EE0FECDCC23
:10122700CD8E07124328E54475F040A4FFAEF09039
:1012370002F812001EE02DFD50010C8C2D8D2E752D
:101247005201021C53900043E0C39402400302136F
:10125700A2900039E0D3954450030213A2E54475E8
:10126700F040A4FFAEF090030212001EE0C3953CCD
:101277005018E54475F040A4FFAEF090030112004A
:101287001EE0F52C752B000213A2E54475F040A46F
:10129700FFAEF090030012001EE0C3953C4003022E
:1012A700133EE54475F040A4FFAEF0900301120031
:1012B7001EE54475F040A4FFAEF0E0FC9002FF127B
:1012C700001EECFEE0FFEEC39FFEE5448E0475F0C2
:1012D70040A4FFAEF090030012001EE0F404253C8A
:1012E7008C0088F0A4FFAEF0E5448F048E0575F0FE
:1012F70040A4FFAEF090030212001EE54475F040D3
:10130700A4FFAEF0E0FA90030012001EEAFEE0FF31
:10131700EEC39FFECDCCCD8E07124328E54475F072
:1013270040A4FFAEF09002FF12001EE02DFD500119
:101337000C8C2B8D2C8064E54475F040A4FFAEF037
:101347009002FF12001EE54475F040A4FFAEF0E0E6
:10135700FC9002FE12001EECFEE0FFEEC39F853CF0
:10136700F0A4FFAEF0E5448F048E0575F040A4FFAE
:10137700AEF090030012001EE0FECDCCCD8E07121A
:101387004328E54475F040A4FFAEF09002FE12003A
:101397001EE02DFD50010C8C2B8D2C755202021C6A
:1013A70053900043E0B4022AE54475F040A4FFAE31
:1013B700F090030112001EE0F52C752B00E5447533
:1013C700F040A4FFAEF09002F812001EE0F52E7573
:1013D7002D00900043E0B4030F90003BE0F52C751F
:1013E7002B00752E00752D00E544B40105755204D8
:1013F7008017E544B40205755205800DE544B40332
:10140700057552068003755203021C53E544D394B5
:10141700034015E54475F040A4FFAEF090030A12AF
:10142700001EE0C3954B4002807DAE23AF24AC2D58
:10143700AD2EEDD39FEC9E401AE54475F040A4FF16
:10144700AEF090030812001EE0A829B80005D39556
:101457002A500280021544E544B54537E544C39553
:101467004F5030E54804D395444028AE23AF24AC11
:101477002BAD2CEFD39DEE9C4019E54475F040A4AD
:10148700FFAEF090030912001EE0A829B8000695E8
:101497002A400280020544C292E54465456008C2BD
:1014A70003754B007551FA755208021C53E544B495
:1014B7000115E54475F040A4FFAEF090030A120051
:1014C7001EE0C3954B40028050A205B34011C205F0
:1014D700754402D206D2047551CD754B008038E5AC
:1014E70044C3954F5031AE23AF24AC2BAD2CEFD373
:1014F7009DEE9C400D900389E0A829B80006952A27
:1015070040028002D205A205B3400C90034AE0C313
:101517009405F54B7551FAC292755207021C53E5B3
:1015270044B40215E54475F040A4FFAEF090030AF9
:1015370012001EE0C3954B40030215CF900033E025
:10154700701DAE23AF24AC2DAD2EEDD39FEC9E4086
:101557000E900388E0A829B80005D3952A50028089
:1015670003754401A205B34009C205754403D204BB
:101577008041E544C3954F503AAE23AF24AC2BAD21
:101587002CEFD39DEE9C4014E548D39401400D9079
:1015970003C9E0A829B80006952A40028002D205AF
:1015A700A205B3400E90038AE0C39402F54B755130
:1015B700FAD204E5446545600D754B00E544B40176
:1015C70005C2047551FAC292755207021C53E544CD
:1015D700B40315E54475F040A4FFAEF090030A127A
:1015E700001EE0C3954B4003021676A205B3400EDA
:1015F700C205754402D206D2047551CD802DAE23A3
:10160700AF24AC2DAD2EEDD39FEC9E400E9003C8BA
:10161700E0A829B80005D3952A5002800ED205907C
:1016270003CAE0C39405F54B7551FAE544C3954FDA
:101637005023E548D39402401CAE23AF24AC2BAD16
:101647002CEFD39DEE9C400D90040AE0A829B8002A
:1016570006952A40028003754404E5446545600DFC
:10166700E544B40405C2037551FA754B00C292757F
:101677005207021C53E54475F040A4FFAEF09003F7
:101687000412001EE0B40117E54475F040A4FFAE54
:10169700F090030A12001EE0241EC3954B4003027C
:1016A700174C753064752F00A203B3500B90004A96
:1016B700E02405C3953C400302174CE54475F04010
:1016C700A4FFAEF090030712001EE0C3953C4064F0
:1016D700E54475F040A4FFAEF090030612001EE546
:1016E7004475F040A4FFAEF0E0FC90030512001E25
:1016F700ECFEE0FFEEC39F853CF0A4FFAEF0E544AF
:101707008F048E0575F040A4FFAEF090030712001A
:101717001EE0FECDCCCD8E07124328E54475F04080
:10172700A4FFAEF090030512001EE02DFD50010C42
:101737008C2F8D30AE23AF24AC2FAD30EFD39DEE81
:101747009C4002D203755209021C53E54475F040D0
:10175700A4FFAEF090030412001EE0B40117E544A5
:1017670075F040A4FFAEF090030A12001EE0240AB1
:10177700C3954B4003021822753064752F00A203EE
:10178700B3500B90004AE02405C3953C4003021870
:1017970022E54475F040A4FFAEF090030712001E47
:1017A700E0C3953C4064E54475F040A4FFAEF0907B
:1017B700030612001EE54475F040A4FFAEF0E0FCFE
:1017C70090030512001EECFEE0FFEEC39F853CF080
:1017D700A4FFAEF0E5448F048E0575F040A4FFAE7C
:1017E700F090030712001EE0FECDCCCD8E0712430A
:1017F70028E54475F040A4FFAEF090030512001EE3
:10180700E02DFD50010C8C2F8D30AE23AF24AC2F73
:10181700AD30EFD39DEE9C4002D203755209021CF6
:1018270053E54BB416037551CDE544B40205A20543
:10183700B34003021947E54BC3940A507D90005CFF
:10184700E0B40258E53C75F00284FF7E0090016A1F
:1018570012001EE0F555E53D75F00A84FF7E009005
:10186700023812001EE0F54DE555254DD39464402E
:101877000BE555254DC39464F5558003755500E573
:101887005575F00284FF7E008F55EFC394335007E0
:10189700EF24CDF55580037555FF801CE53C75F0A9
:1018A7000284FF7E0090016A12001EE075F0028438
:1018B700FF7E00EF24CDF555807B90005CE0B402FD
:1018C70058E53C75F00284FF7E0090019C12001ED3
:1018D700E0F555E53D75F00A84FF7E009002381269
:1018E700001EE0F54DE555254DD39464400BE555B5
:1018F700254DC39464F5558003755500E55575F07E
:101907000284FF7E008F55EFC394335007EF24CD39
:10191700F55580037555FF801CE53C75F00284FF83
:101927007E0090019C12001EE075F00284FF7E008D
:10193700EF24CDF555E54BD394024004C2A0C2066F
:10194700E544B40206A205B3B34002807B90005C75
:10195700E0B40258E53C75F00284FF7E0090019CDC
:1019670012001EE0F555E53D75F00A84FF7E0090F4
:10197700023812001EE0F54DE555254DD39464401D
:101987000BE555254DC39464F5558003755500E562
:101997005575F00284FF7E008F55EFC394335007CF
:1019A700EF24CDF55580037555FF801CE53C75F098
:1019B7000284FF7E0090019C12001EE075F00284F5
:1019C700FF7E00EF24CDF555E544B40307E54BC38F
:1019D70094194003021A6090005CE0B40258E53C99
:1019E70075F00284FF7E0090019C12001EE0F55501
:1019F700E53D75F00A84FF7E0090023812001EE074
:101A0700F54DE555254DD39464400BE555254DC35C
:101A17009464F5558003755500E55575F00284FF0C
:101A27007E008F55EFC394335007EF24CDF55580D3
:101A3700037555FF801CE53C75F00284FF7E00901E
:101A4700019C12001EE075F00284FF7E00EF24CD9A
:101A5700F555E54BB41602C20475520A021C53E54C
:101A670044D394034006E54B640A60028003755132
:101A7700CDE5446402601090003AE02402A823B840
:101A87000005D3952450028002C203E544B401192E
:101A9700A205B35014E53CC39405500D900349E0EB
:101AA700A829B80006952A4002800ED20590034A5D
:101AB700E0C39405F54B7551FA900043E0C39403D6
:101AC700503BE544D394014034E54475F040A4FF0E
:101AD700AEF09002FE12001EE0A823B8001FD395B7
:101AE70024401AE54475F040A4FFAEF090030912B4
:101AF700001EE0A829B80005D3952A50028052E5B8
:101B07004464036015900033E0700415448009E5D0
:101B170044D3940340021544802AA205B350099088
:101B270003CAE0C3954B4002801AE53CC3940550B5
:101B370005754401800ED2059003CAE0C39405F5EC
:101B47004B7551FAE544B40108C203C204C2A0C2EE
:101B57000575520B021C53E544D39401402FE5440D
:101B670075F040A4FFAEF09002FC12001EE0C39592
:101B77003C501AE54475F040A4FFAEF090030812FC
:101B8700001EE0A829B80005D3952A50028033E546
:101B970044B40305A205B34002800ED2059003CAE0
:101BA700E0C39405F54B7551CDE54464036013908C
:101BB7000033E0700415448009E544D394034002E0
:101BC7001544E544D394034021E548C39403501AD0
:101BD700E54475F040A4FFAEF090030812001EE044
:101BE700A829B80005D3952A50028009E544D39463
:101BF7000340021544E544B4031FE548B4011AE560
:101C07004475F040A4FFAEF090030812001EE0A850
:101C170029B80005D3952A5002801AE544B4030574
:101C2700A205B34002800ED2059003CAE0C3940513
:101C3700F54B7551CD90004AE0D3953C5009900083
:0C1C47003EE0C3953C5002C20375520001
:1024A4000210F202124C0213A80214130214B40212
:1024B40015260215D502167C021752021828021A94
:0424C40066021B5E33
:101C5300900043E07003021E8FA2A5B34008A2A424
:101C6300B34003021E78AE31AF327441D39F749CEC
:101C73009E4005783112003FAE31AF32EFB4880693
:101C8300EEB413028003021E53A2A55003021D8269
:101C9300900043E0B4010B900039E0D3954F40022C
:101CA300054F900043E0B40275900039E0D39544AA
:101CB3004019E54475F040A4FFAEF09002FE120017
:101CC3001EE0A823B8000695244002804BE544B4E7
:101CD300010ED20590034AE0C39405F54B7551FA02
:101CE300E544B40207E548D3940150028010D205BD
:101CF30090038AE0C39405F54B7551FAD204E54489
:101D0300D394024007E548D394025002800A054465
:101D1300C203754B007551FA900039E0F54F9000FE
:101D230043E0B4035A900039E0D39544404BE54473
:101D3300B4010ED20590034AE0C39405F54B7551E7
:101D4300FAE544B40207E548D3940150028013D264
:101D53000590038AE0C39405F54B7551FAD20475D7
:101D63004B00E544D394024007E548D39402500264
:101D730080070544C2037551FA900039E0F54FA27C
:101D8300A45003021E53900043E0B40150E544D332
:101D930094014046E54475F040A4FFAEF09003087B
:101DA30012001EE0A829B8002CD3952A4027E54449
:101DB300B40313D2059003CAE0C39405F54B7551E0
:101DC300FA754F02800D154485444F7551FA754BD2
:101DD30000C204800385444F8003754F0190004384
:101DE300E0D39401405EE544D394014034E5447567
:101DF300F040A4FFAEF09002FB12001EE0A823B84F
:101E0300001FD39524401AE54475F040A4FFAEF0BB
:101E130090030812001EE0A829B80005D3952A50A4
:101E2300028021E544B40310D2059003CAE0C394B1
:101E330005F54B7551FA800C15447551FA754B0035
:101E4300C203C204E548B40704054E8003754E007F
:101E530090006BE0B4010EAE31AF32EF6440700519
:101E6300EE649C6002800EA2A54003754901A2A402
:101E73004003754902A2A5B3B35006A2A4B3B3406D
:101E8300028006753200753100021F90A2A5B3408F
:101E930008A2A4B34003021F7CAE31AF327441D316
:101EA3009F749C9E4005783112003FAE31AF32EFF4
:101EB300B48806EEB413028003021F7CA2A5406F10
:101EC300900052E0605A900034E0B401079000346F
:101ED300E4F080069000347401F0900034E0700563
:101EE300754F048003754F05900034E0B40104D2AC
:101EF300A18002C2A1E544B4051AE54475F040A4EB
:101F0300FFAEF090030812001EE0A829B80005D325
:101F1300952A50028008754404C203754B00800360
:101F2300754F05E548B40704054E8003754E00A2BE
:101F3300A44046900053E06034900033E0B40107BE
:101F4300900033E4F080069000337401F090003386
:101F5300E0B40117D2A2E544B4010ED20590034ABE
:101F6300E0C39405F54B7551FA8002C2A2E548B46B
:101F73000704054E8003754E00A2A5B3B35006A215
:101F8300A4B3B340028006753200753100E549659C
:101F93004A600690006CE06002802CE5499024C8FA
:101FA300F82828738012122C66800D122D51800898
:081FB300122E3C8003122F27BF
:0F24C800021FA7021FA9021FAE021FB3021FB8F7
:101FBB001200881202BC85494A741B900024F0E57C
:101FCB0048C394065005E544B54503022060C2039F
:101FDB00E54475F040A4FFAEF090030C12001EE038
:101FEB0030E003D38001C39296E54475F040A4FF23
:101FFB00AEF090030D12001EE030E003D38001C35E
:10200B009295E54475F040A4FFAEF090030E1200DC
:10201B001EE030E003D38001C392A0E54475F0408D
:10202B00A4FFAEF090030F12001EE030E003D3804C
:10203B0001C39297A206B34002D2A0854445AE29B4
:10204B00AF2A7405BE00039F5007E53CD39405509F
:10205B00028002D292E548D3940550030221ADC20F
:10206B0003E544D394015003022102E54475F0408B
:10207B00A4FFAEF090030812001EE0A829B80007D9
:10208B00D3952A40021544E54465456067E54475E0
:10209B00F040A4FFAEF090030C12001EE030E00302
:1020AB00D38001C39296E54475F040A4FFAEF09047
:1020BB00030D12001EE030E003D38001C39295E5BF
:1020CB004475F040A4FFAEF090030E12001EE030FA
:1020DB00E003D38001C392A0E54475F040A4FFAEAA
:1020EB00F090030F12001EE030E003D38001C39287
:1020FB00978544450221ADE548B40634900096E03F
:10210B0030E003D38001C39296900097E030E00358
:10211B00D38001C39295900098E030E003D3800107
:10212B00C392A0900099E030E003D38001C3929753
:10213B00E548B4073490008FE030E003D38001C34F
:10214B009296900090E030E003D38001C39295907B
:10215B000091E030E003D38001C392A0900092E0A5
:10216B0030E003D38001C39297E548B40834900064
:10217B0088E030E003D38001C39296900089E03071
:10218B00E003D38001C3929590008AE030E003D343
:10219B008001C392A090008BE030E003D38001C399
:1021AB009297E54864066005E548B40808E5B54430
:1021BB0010F5B58006E5B554EFF5B5E53C75F002C5
:1021CB0084FF7E0090013812001EE075F00284FF40
:1021DB007E00EF24CDF54CE595C3954C4004C2939E
:1021EB008002D293A204B34002800FA203B3400734
:1021FB00E548D3940540037555CDE595C3955540FA
:10220B0004C2948002D294E595C395514004C291C7
:10221B008002D291E56CC3940D501DE56C75F002F4
:10222B0084AFF07E00EF4E70051237AF800AA2ED3F
:10223B00B34005C2ED1237AFE54ED3940450030201
:10224B00236F75CF01C293AE31AF327488D39F74B5
:10225B00139E4005A2A5B34014AE31AF327488D3A0
:10226B009F74139E4005A2A4B3400280587831128C
:10227B00003FAE31AF32EFB4884BEEB41347A2A59B
:10228B00B35009900039E0D395445002800C0544BB
:10229B00E544B402037544038011A2A5B350089022
:1022AB000039E0654460028002D203A2A4B3500758
:1022BB00E544D394015002800C1544E544B4020369
:1022CB00754401C203A2A5B3B35006A2A4B3B34095
:1022DB00028006753200753100E54465456069E59D
:1022EB004475F040A4FFAEF090030C12001EE030DA
:1022FB00E003D38001C39296E54475F040A4FFAE92
:10230B00F090030D12001EE030E003D38001C39266
:10231B0095E54475F040A4FFAEF090030E12001E3D
:10232B00E030E003D38001C392A0E54475F040A4F4
:10233B00FFAEF090030F12001EE030E003D38001DC
:10234B00C39297C294854445A20340057555CD8031
:10235B00037555FFE595C395554004C2948002D291
:10236B009402224DA20CB3500DAE25AF2674E8C3D8
:10237B009F74039E4002800575FFA0D20CAE25AF63
:10238B0026EFD39420EE944E500302246F1205FBDC
:10239B00C28E758D00758B00754100D28EC2037590
:1023AB0054007553007555CD754405752400752380
:1023BB0000754600754B00C287900043E06004D265
:1023CB00908002C290900034E0B40104D2A180024C
:1023DB00C2A1900033E0B40104D2A28002C2A2A237
:1023EB0008B34008E5B54440F5B58006E5B554BFE4
:1023FB00F5B5900055E060077401F508123569904A
:10240B000058E060077402F508123569E548B40717
:10241B0008E5B54480F5B58006E5B5547FF5B59074
:10242B00000474FDF0A374E8F0E56CB40D03756C57
:10243B0000752600752500758D00758B00754100A4
:10244B00900025E0C394035008900025E004F08031
:10245B00067403900025F0900025E0B40306E5B563
:10246B0054FEF5B5AE27AF28EFD39410EE9427406A
:10247B001CC2CA75CD0075CC00752800752700D21B
:10248B00CA754300752A00752900754700020D3087
:10425700000001000132016401960196020002127A
:1042670002240200020003000340038003C004008D
:104277000440048004C0050006000600060006008E
:10428700060006000600060000FF013101630195E4
:1042970001FF01FF0211022302FF02FF02FF033F9A
:1042A700037F03BF03FF043F047F04BF04FF05FF31
:1042B70006FF06FF06FF06FF06FF06FF06FF06FFCF
:1024D700900041E090083BF0900048E090083CF005
:1024E700900049E090083DF090004CE090083EF0E5
:1024F70090004DE090083FF0900050E0900840F0C9
:10250700900051E0900841F090005CE0900842F0A4
:1025170090005EE0900843F0900062E0900844F07D
:10252700900064E0900845F0900065E0900846F060
:10253700900066E0900847F0900067E0900848F048
:1025470090006AE0900849F090006BE090084AF02C
:1025570090006DE090084BF090006EE090084CF012
:1025670090007AE090084DF090007BE090084EF0E4
:1025770090007CE090084FF090007DE0900850F0CC
:1025870090007EE0900851F090007FE0900852F0B4
:10259700900080E0900853F0900081E0900854F09C
:1025A700900083E0900855F0900084E0900856F082
:1025B700900085E0900857F0900086E0900858F06A
:1025C700900124E0900859F0900125E090085AF016
:1025D700900126E090085BF022900838E4F0A3F021
:1025E700755C00755B00756600756700C20DD20EDD
:1025F700756000755F0075623C756100756D0075EB
:102607006E00756B0022750B00750A00AE0AAF0BE2
:10261700AC08AD09EDC39FEC9E401674FF1243183A
:1026270075CF01780B740126F6500418E436F6507E
:10263700DB22C2AF75D900758F0375B7A575B7F1E2
:1026470090F800E4F0758F0175B7A575B7F1E556F9
:1026570090F800F075B7A575B7F190F801E4F0753B
:10266700B7A575B7F1900877E090F802F075B7A5B0
:1026770075B7F190087BE090F803F075B7A575B7CB
:10268700F1900878E090F804F075B7A575B7F19068
:102697000879E090F805F075B7A575B7F190087A55
:1026A700E090F806F075B7A575B7F190087CE09053
:1026B700F807F0758F0075D940D2AF2290083AE03D
:1026C700B4AB61C2AF75D90075B62275F522758FA7
:1026D7000375B7A575B7F1740090F600F0758F0113
:1026E700755800755700AE57AF58743BBE00279F0B
:1026F700402475B7A575B7F190083B12001EE0FCA2
:1027070090F60012001EECF07858740126F650047B
:1027170018E436F650D0758F0075F51175B620752B
:10272700D940D2AF22C2AF75D90075F522755800CE
:10273700755700AE57AF58743BBE00229F401F909D
:10274700F60012001EE493FC90083B12001EECF00A
:102757007858740126F6500418E436F650D575F506
:102767001175D940D2AF2290083AE0B4AA0280038B
:102777000228ABC2AF75D90075B62275F522758FE1
:102787000375B7A575B7F1740090EE00F075B7A59E
:1027970075B7F1740090F000F075B7A575B7F174CF
:1027A7000090F200F075B7A575B7F1740090F400CA
:1027B700F0758F01755800755700AE57AF5874FF05
:1027C700C39F74019E402475B7A575B7F190003873
:1027D70012001EE0FC90EE0012001EECF078587418
:1027E7000126F6500418E436F650CF755800755791
:1027F70000AE57AF5874FFC39F74019E402475B74E
:10280700A575B7F190023812001EE0FC90F0001297
:10281700001EECF07858740126F6500418E436F6DA
:1028270050CF755800755700AE57AF5874FFC39F08
:1028370074019E402475B7A575B7F190043812004E
:102847001EE0FC90F20012001EECF078587401268E
:10285700F6500418E436F650CF755800755700AE99
:1028670057AF5874FFC39F74019E402475B7A57571
:10287700B7F190063812001EE0FC90F40012001E1B
:10288700ECF07858740126F6500418E436F650CF69
:10289700758F0075F51175B62075D940D2AF743AAA
:1028A700900738F02290083AE0B4AA028003022980
:1028B700E9C2AF75D90075B62275F522758F037514
:1028C700B7A575B7F1740090E600F075B7A575B7B1
:1028D700F1740090E800F075B7A575B7F174009032
:1028E700EA00F075B7A575B7F1740090EC00F075C4
:1028F7008F01755800755700AE57AF5874FFC39FC7
:1029070074019E402475B7A575B7F1900038120081
:102917001EE0FC90E60012001EECF07858740126C9
:10292700F6500418E436F650CF755800755700AEC8
:1029370057AF5874FFC39F74019E402475B7A575A0
:10294700B7F190023812001EE0FC90E80012001E5A
:10295700ECF07858740126F6500418E436F650CF98
:10296700755800755700AE57AF5874FFC39F740171
:102977009E402475B7A575B7F190043812001EE084
:10298700FC90EA0012001EECF07858740126F6500D
:102997000418E436F650CF755800755700AE57AF98
:1029A7005874FFC39F74019E402475B7A575B7F18E
:1029B70090063812001EE0FC90EC0012001EECF0AE
:1029C7007858740126F6500418E436F650CF758F00
:1029D7000075F51175B62075D940D2AF743A9007D6
:1029E70038F02290083AE0B4AA028003022B27C2EB
:1029F700AF75D90075B62275F522758F0375B7A522
:102A070075B7F1740090DE00F075B7A575B7F1746E
:102A17000090E000F075B7A575B7F1740090E2007B
:102A2700F075B7A575B7F1740090E400F0758F01E4
:102A3700755800755700AE57AF5874FFC39F7401A0
:102A47009E402475B7A575B7F190003812001EE0B7
:102A5700FC90DE0012001EECF07858740126F65048
:102A67000418E436F650CF755800755700AE57AFC7
:102A77005874FFC39F74019E402475B7A575B7F1BD
:102A870090023812001EE0FC90E00012001EECF0ED
:102A97007858740126F6500418E436F650CF755866
:102AA70000755700AE57AF5874FFC39F74019E401F
:102AB7002475B7A575B7F190043812001EE0FC9095
:102AC700E20012001EECF07858740126F650041844
:102AD700E436F650CF755800755700AE57AF5874A7
:102AE700FFC39F74019E402475B7A575B7F1900683
:102AF7003812001EE0FC90E40012001EECF078583B
:102B0700740126F6500418E436F650CF758F007519
:102B1700F51175B62075D940D2AF743A900738F0E1
:102B27002290083AE0B4AA028003022C65C2AF756E
:102B3700D90075B62275F522758F0375B7A575B7D8
:102B4700F1740090D600F075B7A575B7F1740090D1
:102B5700D800F075B7A575B7F1740090DA00F07575
:102B6700B7A575B7F1740090DC00F0758F01755843
:102B770000755700AE57AF5874FFC39F74019E404E
:102B87002475B7A575B7F190003812001EE0FC90C8
:102B9700D60012001EECF07858740126F65004187F
:102BA700E436F650CF755800755700AE57AF5874D6
:102BB700FFC39F74019E402475B7A575B7F19002B6
:102BC7003812001EE0FC90D80012001EECF0785876
:102BD700740126F6500418E436F650CF7558007580
:102BE7005700AE57AF5874FFC39F74019E402475BA
:102BF700B7A575B7F190043812001EE0FC90DA0013
:102C070012001EECF07858740126F6500418E436CA
:102C1700F650CF755800755700AE57AF5874FFC3BD
:102C27009F74019E402475B7A575B7F190063812B9
:102C3700001EE0FC90DC0012001EECF078587401D6
:102C470026F6500418E436F650CF758F0075F51147
:102C570075B62075D940D2AF743A900738F022C2C2
:102C6700AF75D90075F522755800755700AE57AF87
:102C77005874FFC39F74019E401F90EE0012001E00
:102C8700E493FC90003812001EECF078587401268B
:102C9700F6500418E436F650D4755800755700AE50
:102CA70057AF5874FFC39F74019E401F90F00012E6
:102CB700001EE493FC90023812001EECF078587462
:102CC7000126F6500418E436F650D47558007557A7
:102CD70000AE57AF5874FFC39F74019E401F90F218
:102CE7000012001EE493FC90043812001EECF078EA
:102CF70058740126F6500418E436F650D475580077
:102D0700755700AE57AF5874FFC39F74019E401F9D
:102D170090F40012001EE493FC90063812001EEC9B
:102D2700F07858740126F6500418E436F650D47536
:102D3700F51175D940D2AF740090006CF074019012
:102D47000042F0743A900738F022C2AF75D9007587
:102D5700F522755800755700AE57AF5874FFC39FDB
:102D670074019E401F90E60012001EE493FC900041
:102D77003812001EECF07858740126F6500418E457
:102D870036F650D4755800755700AE57AF5874FFD4
:102D9700C39F74019E401F90E80012001EE493FC3D
:102DA70090023812001EECF07858740126F6500491
:102DB70018E436F650D4755800755700AE57AF581B
:102DC70074FFC39F74019E401F90EA0012001EE427
:102DD70093FC90043812001EECF07858740126F624
:102DE700500418E436F650D4755800755700AE579E
:102DF700AF5874FFC39F74019E401F90EC001200F0
:102E07001EE493FC90063812001EECF0785874010B
:102E170026F6500418E436F650D475F51175D940E6
:102E2700D2AF740090006CF07402900042F0743AD4
:102E3700900738F022C2AF75D90075F52275580092
:102E4700755700AE57AF5874FFC39F74019E401F5C
:102E570090DE0012001EE493FC90003812001EEC76
:102E6700F07858740126F6500418E436F650D475F5
:102E77005800755700AE57AF5874FFC39F74019E33
:102E8700401F90E00012001EE493FC9002381200ED
:102E97001EECF07858740126F6500418E436F65004
:102EA700D4755800755700AE57AF5874FFC39F7459
:102EB700019E401F90E20012001EE493FC9004382C
:102EC70012001EECF07858740126F6500418E43608
:102ED700F650D4755800755700AE57AF5874FFC3F6
:102EE7009F74019E401F90E40012001EE493FC9023
:102EF700063812001EECF07858740126F6500418B4
:102F0700E436F650D475F51175D940D2AF740090F8
:102F1700006CF07403900042F0743A900738F02286
:102F2700C2AF75D90075F522755800755700AE57B1
:102F3700AF5874FFC39F74019E401F90D6001200C4
:102F47001EE493FC90003812001EECF078587401D0
:102F570026F6500418E436F650D475580075570015
:102F6700AE57AF5874FFC39F74019E401F90D8009F
:102F770012001EE493FC90023812001EECF0785801
:102F8700740126F6500418E436F650D475580075C7
:102F97005700AE57AF5874FFC39F74019E401F90F0
:102FA700DA0012001EE493FC90043812001EECF0C5
:102FB7007858740126F6500418E436F650D475583C
:102FC70000755700AE57AF5874FFC39F74019E40FA
:102FD7001F90DC0012001EE493FC90063812001EBE
:102FE700ECF07858740126F6500418E436F650D4FD
:102FF70075F51175D940D2AF740090006CF0740468
:10300700900042F0743A900738F022E56764046054
:1030170006E59964FF60028031A20D4004D20D805D
:1030270027E567600874E62567900024F0E5666089
:103037000874F02566900024F0E567B4010280FE6D
:10304700756700756600C20D8002C20DE567903D89
:103057004CF8282873756700E599B4FF0375660176
:10306700E599B4FE03756602E599B4FD0375660339
:10307700E599B4FC03756604E599B4FA037566052A
:10308700E599B4FB067567011205FBE599B4F906E6
:103097007567041205FBE599B4F7411205FBC29C5D
:1030A70074AB90083AF01226C374AA90083AF0E578
:0130B70049CF
:033D4C0002305CE6
:1030B800903DACF8282873801212276E800D1228D4
:0B30C800AC80081229EA8003122B28BC
:0F3DAC000230BF0230C10230C60230CB0230D02D
:1030D30090083AE4F0D29C7567007566007599F71D
:1030E300E599D394E54007E599C394F0400280162F
:1030F3008599687567027E017F00E568C394E612CF
:1031030043468E5D8F5E900838E4F0A3F0E599D3D3
:1031130094C44007E599C394E640028028859968E2
:1031230075670374E5C39568F55E755D00AE5DAFC5
:103133005E90425712002EE493F87401939008387E
:10314300C8F0A3C8F0D299023427900838E0FEA350
:10315300E0FF90003812001EE599F0900838120045
:103163000E900838E0FEA3E0FFEFB40106EEB407CB
:10317300028003023235900738E0B43C0280030238
:10318300323512099AA209B35005A20AB34002804C
:1031930053C29C1200881202BC900124E09008598B
:1031A300F0900125E090085AF0900126E090085B2A
:1031B300F074AB90083AF01226C374AA90083AF060
:0231C300E549DC
:033D4F0002314DF1
:1031C500903DBBF8282873801212276E800D1228B7
:0B31D500AC80081229EA8003122B28AE
:0F3DBB000231CC0231CE0231D30231D80231DDD8
:1031E00090083AE4F08043C29C1224D774009008FF
:1031F00059F0740090085AF0740090085BF074ABBA
:1032000090083AF01226C374AA90083AF012276E7A
:103210001228AC1229EA122B28D29C7599FB7464EF
:10322000F50975080012260D80FED29C75670075A1
:1032300066007599FB023427900838E0FEA3E0FF92
:10324000EF4E700685995C755B00900838E0FEA330
:10325000E0FF74016F4E701BAC5BAD5CAA5DAB5EB2
:10326000ED2BFBEC3AFA8A068B0790003812001E11
:10327000E599F090083812000E900838E0FEA3E0BF
:10328000FF74026F4E700C1202BC8568997567005E
:10329000756600023427900838E0FEA3E0FF900036
:1032A0003812001EE599F090083812000E90083888
:1032B000E0FEA3E0FFAC5DAD5E8F028E038C068D59
:1032C0000790428F12002EE493F9740193FEEAD323
:1032D0009EEB994009856899756700756600023410
:1032E00027900838E0FEA3E0FF90003812001EE5AA
:1032F00099F090083812000E900838E0FEA3E0FF25
:10330000EFB40006EEB401028003023427900018E7
:10331000E0D394C7400B900018E0C394C8F56980CF
:103320001A900018E0D39463400B900018E0C39407
:1033300064F5698006900018E0F569E56975F002AA
:10334000A4FFAEF08F65EF90003812435EEFFCE013
:10335000FDEC90003B12435EEDFCE0FDEC2DB56909
:103360000280030234180FEF90003812435EE565C7
:10337000FFE0FCEF90003C12435EECFFE0FCEFC38B
:103380009CB569028003023418E56590003A124347
:103390005EE565FFE0FCEF90003D12435EECFFE070
:1033A000FCEF2CB56972E56590003E12435EE0C308
:1033B0009569900877F0E56590003F12435EE0C3A1
:1033C0009569900878F0E56590004212435EE0C38D
:1033D0009569900879F0E56590004312435EE0C37B
:1033E000956990087AF0E56590004412435EE0C369
:1033F000956990087BF0E56590004512435EE0C357
:10340000956990087CF01226397599F97464F5096C
:1034100075080012260D80FE7599FF7464F5097514
:07342000080012260D80FEDA
:093D52000232380232960232E11D
:1034270022E566903D5BF8282873023568900838D6
:10343700E0FEA3E0FF90000812001EE0F599900857
:103447003812000E900838E0FEA3E0FF741C6F4EA0
:1034570070037566000235688550990235689008D3
:1034670038E0FEA3E0FF90003812001EE0F599EF68
:10347700B40107EEB4070375660090083812000E12
:07348700023568900839E0EE
:0F3D5B0002343102343402345F02346502348A98
:10348E00903DCAF828287385249902355D852A99BE
:10349E0002355D853B9902355D853D9902355D8529
:1034AE00449902355D854F9902355D8548990235FF
:1034BE005D85499902355D756A00900053E070068E
:1034CE00900052E060028016A2A44006E56A440411
:1034DE00F56AA2A54006E56A4402F56A801A9000D4
:1034EE0034E0B40106E56A4410F56A900033E0B4A6
:1034FE000106E56A4420F56AA203B34006E56A4474
:10350E0001F56AA208B34006E56A4408F56A856AC1
:10351E0099803CA20EB340077599FAC20E8017A28D
:10352E000BB3400575990F800B900024E0F5999030
:10353E000024E4F0C20B8017853A998012854099D9
:0F354E00800D856B9980087599FC800375660068
:103DCA0002349502349B0234A10234A70234AD02B4
:103DDA0034B30234B90234BF0234C5023521023584
:0D3DEA004602354B02355002355502355A60
:0B355D0090083812000E800312023BA1
:033D6A00023565BA
:1035680022E50875F003A4FFAEF0EF241AF509E58B
:103578000904F50AE5092402F50BE509900038125B
:10358800435EE0903D6DF828287380218524638090
:103598001C852A638017853B638012853D63800DF7
:0D35A800854463800885486380038549637E
:103D6D0002359202359402359902359E0235A30231
:083D7D0035A80235AD0235B294
:1035B500E50A90003812435EE50BFEE0FFEE900051
:1035C5003812435EEFFEE0FFEED39F40030236C3A1
:1035D500E50990003812435EE0D394044051E50AB2
:1035E50090003812435EE0D39563500EE50B9000D2
:1035F5003812435EE0C395635002800AE508F50C76
:10360500D39210120048E50A90003812435EE0D3C9
:103615009563500EE50B90003812435EE0C3956349
:10362500500AE508F50CC392101200480236C0E5B1
:103635000990003812435EE0B40432E50B9000387F
:1036450012435EE0C39563500AE508F50CD392106A
:10365500120048E50A90003812435EE0D3956340B6
:103665000AE508F50CC39210120048804EE50A9051
:10367500003812435EE0C39563500EE50B900038A9
:1036850012435EE0D395635002800AE508F50CD33A
:103695009210120048E50A90003812435EE0D39577
:1036A50063500EE50B90003812435EE0C3956350FE
:1036B5000AE508F50CC392101200480237AEE50979
:1036C50090003812435EE0D394044051E50A90001F
:1036D5003812435EE0C39563400EE50B9000381247
:1036E500435EE0D395634002800AE508F50CC3927A
:1036F50010120048E50A90003812435EE0C3956356
:10370500400EE50B90003812435EE0D39563400A06
:10371500E508F50CD392101200480237AEE5099082
:10372500003812435EE0B40432E50A9000381243D3
:103735005EE0C39563500AE508F50CC392101200CC
:1037450048E50B90003812435EE0D39563400AE5E7
:1037550008F50CD39210120048804EE50A90003807
:1037650012435EE0C39563400EE50B9000381243AB
:103775005EE0D39563400AE508F50CD3921012007C
:1037850048E50A90003812435EE0D39563400EE5A4
:103795000B90003812435EE0C395634002800AE552
:1037A50008F50CC3921012004822E56C903D85F88F
:1037B500282873023D397E017F00E5BE124346E5A8
:1037C500BD2FFF50010E8E598F5A900064E0B40151
:1037D5000F7E0F7FFFAC59AD5A1200038E598F5AD9
:1037E500900063E0B40245AE59AF5A900000E0FC8A
:1037F500A3E0FDEDD39FEC9E400A900000E559F053
:10380500A3E55AF0AE59AF5A900002E0FCA3E0FDE3
:10381500EFD39DEE9C400A900002E559F0A3E55ACE
:10382500F0AE59AF5A74041243388F3B900063E0F1
:103835007058AE59AF5A900000E0FCA3E0FDEFD3FD
:103845009DEE9C40091200038E598F5A8006755AC9
:1038550000755900900062E0700674FF900062F0F8
:10386500AE59AF5A7410124346900062E08E048F31
:1038750005FF1243288C598D5A7400D39D74019C01
:103885004005855A3B8003753BFFE53B75F00AA46F
:10389500FFAEF074198E048F05FF1243288D3CEDA1
:1038A5002560FFAE5F50010E74011243388F3C85D1
:1038B5003C60755F00EFD394624003753C629000F5
:1038C5005CE07006900050E060028006756C0502B1
:1038D50037AF75BB17023D39023D397E017F00E5E3
:1038E500BE124346E5BD2FFF50010E8E598F5A90EB
:1038F500005CE0B4017AE56245616025AC61AD62CA
:103905001DBDFF011C8F028E038C068D07903DF7B0
:1039150012002EE493FE740193FFEFC39AEE9B40D1
:103925000280057861124370AE61AF6274B3BE0068
:1039350021D39F401DAC59AD5A0FBF00010E903DDC
:10394500F712002EE493FE740193FFEDC39FEC9EE6
:1039550040028005786112003FAE61AF6290005E63
:10396500E012434674648E048F05FF1243288D3D93
:10397500E56FB40129AE59AF5AEFD39400EE940820
:10398500400F900050E0B40104C2088002D20880C4
:103995000D900050E0B40104D2088002C20875BB46
:1039A50016023D39023D397E017F00E5BE124346D0
:1039B500E5BD2FFF50010E8E598F5A90005CE0B483
:1039C500027AE56245616025AC61AD621DBDFF010E
:1039D5001C8F028E038C068D07903F6112002EE42A
:1039E50093FE740193FFEFC39AEE9B400280057826
:1039F50061124370AE61AF6274B3BE0021D39F40C4
:103A05001DAC59AD5A0FBF00010E903F6112002E3B
:103A1500E493FE740193FFEDC39FEC9E4002800585
:103A2500786112003FAE61AF6290005EE0124346DE
:103A350074648E048F05FF1243288D3DE56FB40233
:103A450029AE59AF5AEFD39400EE9408400F900079
:103A550050E0B40104C2088002D208800D900050E5
:103A6500E0B40104D2088002C20890005CE0700353
:103A7500753D00900050E07002C20875BB1F023D05
:103A850039023D397E017F00E5BE124346E5BD2F73
:103A9500FF50010E8E598F5A740912434674E68EF3
:103AA500048F05FF1243288C398D3AE56D2DFD50A5
:103AB500010C74018C068D071243388E398F3A85B7
:103AC5003A6D75BB19023D39023D397E017F00E52E
:103AD500BE124346E5BD2FFF50010E8E598F5A7415
:103AE500041243388F4090006AE0B401028003025B
:103AF5003BA6756500756500E565D394074003022F
:103B05003B9CE56590002B12435EE0D39540501A2F
:103B1500E56590002B12435EE0F4042540FEE56563
:103B250090087D12435EEEF08017E56590002B123C
:103B3500435EE0C39540FEE56590087D12435EEE69
:103B4500F0E565C39404400990006EE0C3956550A7
:103B55003BE5656029E56590087D12435EFEE0FF63
:103B6500EE900885E0D39F4013E56590087D1243EC
:103B75005EE0900885F0E565900886F0800E900877
:103B85007DE0900885F07400900886F078657401F2
:103B950026F64003023AFD900886E0F4042408F571
:103BA5004890006AE0D394014033E540D3946E40D9
:103BB50004D20F8002C20F75480590006AE0B40276
:103BC50005A20FB34002800375480790006AE0B470
:103BD5000306A20FB3B340028003754807E56E657F
:103BE500486008E54404F54585486EE548B407088E
:103BF500E5B54480F5B58006E5B5547FF5B5E548EE
:103C050064066005E548B40808E5B54410F5B580D7
:103C150006E5B554EFF5B575BB13023D39023D39DF
:103C25007E017F00E5BE124346E5BD2FFF50010E24
:103C35008E598F5A74041243388F6B90006BE0B421
:103C450002028003023D34756500756500E565D3A4
:103C550094034003023CE1E56590002712435EE0D2
:103C6500D3956B501AE56590002712435EE0F40486
:103C7500256BFEE56590088712435EEEF08017E53B
:103C85006590002712435EE0C3956BFEE5659008DD
:103C95008712435EEEF0E5656029E56590088712B9
:103CA500435EFEE0FFEE90088BE0D39F4013E56591
:103CB50090088712435EE090088BF0E56590088CCC
:103CC500F0800E900887E090088BF0740090088CC7
:103CD500F07865740126F64003023C5290006CE0D2
:103CE500704DE52A45296036E549C39403500A908D
:103CF500088CE004C394034002800790088CE0041C
:103D0500F549E549D39402400A90088CE004D39420
:103D1500025002800790088CE004F5498011900854
:103D25008CE004F549E549D39404400375490175D0
:043D3500BB18800037
:103D85000237B80237BB0238DD0238E00239A90232
:103D950039AC023A86023A89023ACD023AD0023C5F
:073DA50022023C25023D391A
:103D3900E56C75F00284AFF07E00EF4E7002D2ECB4
:033D4900056C22E4
:09435E002582F58250020583223C
:10002E00EF2F500205832582F582E5833E2EF58360
:01003E00229F
:08000300C3EF9DFFEE9CFE22FD
:08003F000806B60002180622B3
:0D000E00A3E004F07006124354E004F02259
:084370000816B6FF0218162220
:0E433800048007C3CE13CECF13CFD5E0F622FC
:10417600BC000FBE0008ED8FF084FFADF022E4FE18
:10418600FF22BE000DEF60FE54F0606F20E70302D1
:10419600422CEAC0E0EBC0E078017A0075F001EE4F
:1041A60020E710EF25E0FFEE33FE0AC5F023C5F049
:1041B60030E7F0EA5407F9096A7A007B00600108E3
:1041C600C3EC9E40167004ED9F4010ED9FFDEC9EE3
:1041D600FCE5F0CA4ACA03F5F08005E5F003F5F000
:1041E600C3EE13FEEF13FFD9D77908CACBCAD8D0CE
:1041F600EAFEEBFFD0E0FBD0E0FA22EC8FF084FC85
:10420600ED54F045F0C48FF084FEEDC454F045F053
:10421600C48FF084FDEEC4FE54F02DFFEE540F3C27
:10422600FEADF07C0022790078008FF0EC7E08204D
:10423600E70DC3CD33CD33C933C9C833C8DEF084E7
:1042460049F9E5F08FF0BE00E6FD7C00E9FFE8FEE7
:014256002245
:0E434600F88FF0A4FFE5F0CE88F0A42EFE2242
:10431800600D782B024322007830D8FED5E0F822D1
:10432800EEC0E07E00124176EFFDEEFCD0E0FE220A
:03000B000242C7E7
:03001B000242E2BC
:03002B000242FD91
:0300000002436751
:0943670075817075D0000209C8CF
:0B001E00E5822FF582E5833EF583228A
:0A4354000582D5820215831582222E
:1042C700C0E0C0F0C083C082C0D075D0001209BD65
:1042D700D0D0D082D083D0F0D0E032C0E0C0F0C0E0
:1042E70083C082C0D075D0001209C0D0D0D082D090
:1042F70083D0F0D0E032C0E0C0F0C083C082C0D02D
:1043070075D0001209C3D0D0D082D083D0F0D0E0CE
:014317003273
:00000001FF
